:1000000012C0189518951895189518951895189563
:10001000189518951895B1C1DBC1189518951895C4
:100020001895189518958FE58DBFC8E3E0E24E2E20
:1000300084E08EBFD4E0F4E05F2EA89584B7082E4C
:10004000877F84BF88E1992781BD91BDEEEFF3E002
:10005000A0E6B0E088278D933197E9F7FDD06624BC
:100060008CE042D1F1D0579AE0E8F0E088E43CD14E
:1000700058E0C895802D32D131965A95D1F704C0F9
:100080000C12120C2020202078948E9A969A8CEDD7
:1000900095E056D1A6E6B1E0BA93AA93A7E6B1E0FF
:1000A000BA93AA931ED02496CFD0ECE2F5E0C4D048
:1000B000A8E0B4E0E6E6F1E0CCD1B6D081E00ED124
:1000C000E4E3F5E0B9D0BED0E6E3F5E0B5D0A8E0D2
:1000D000B4E0E7E6F1E0BDD1A7D0EEE3F5E0ACD0C7
:1000E000D6CF80E080939C01AAE6B1E088278C936C
:1000F0008E9A969889E190E023D1969AEF93FF9398
:10010000ECE9F0E011D1FF91EF918E98EF93FF931E
:10011000ECE9F0E009D1FF91EF91869B05C081E009
:10012000A881B9818C9378C0EF93FF93ECE3F1E061
:10013000FBD0FF91EF91869905C082E0A881B9813B
:100140008C936AC0869B01C0FDCF869901C0FDCF0C
:10015000EF93FF93E4E7F0E0E7D0FF91EF91869B08
:100160000AC0AAE6B1E059D0E0E4F5E0FDD0869BF4
:1001700001C0FDCF06C0AAE6B1E04FD0E2E4F5E051
:10018000F3D0ACE9B1E08C918F5F8C9300919C012E
:10019000083209F0DACF8E9A969AEAE6F1E008E0A2
:1001A000A3E9B1E0B5D1A3E9B1E099D1A881B981C2
:1001B0000C9381E1EAE6F1E008E00A93A3E9B1E0FB
:1001C000A0D1A3E9B1E08BD1AA81BB810C93AAE6AF
:1001D000B1E0A6D1EA2FFB2F39970FEFA3E9B1E0E9
:1001E00097D1A3E9B1E07BD1A8E6B1E00C93AA8155
:1001F000BB810C91A881B9814C91040FA9E6B1E0B3
:100200000C934091680100916901041709F404C03E
:1002100083E0A881B9818C9308958F938D91882371
:10022000E9F711978F910895A8E0B4E08D918823A4
:1002300011F054D0FBCF08959CD0802D11F04ED0FA
:10024000FBCF089580EC50C081E04ED002D080E812
:100250004BC083E0992774C08AEF90E071D0A09AD8
:10026000A19AA29AA39AA49AA59AAD9885E090E043
:1002700067D0AC98A898A998AA9AAB9AAC9AEF9331
:10028000FF93ECE8F1E050D0FF91EF91AC9855D09E
:10029000AC9AEF93FF93ECE8F1E046D0FF91EF9139
:1002A000AC984BD0AC9AEF93FF93ECE8F1E03CD0E4
:1002B000FF91EF91AC9841D0AB98AC9AEF93FF933C
:1002C000ECE8F1E031D0FF91EF91AC9836D088E2C4
:1002D0000BD08EE009D086E007D00895AD9A8295C4
:1002E00005D004D02AD00895AD98F9CF859510F4A3
:1002F000AB9A01C0AB98859510F4AA9A01C0AA9850
:10030000859510F4A99A01C0A998859510F4A89A2A
:1003100001C0A898AC9AEF93FF93ECE8F1E004D009
:10032000FF91EF91AC9808953197F1F70895689493
:1003300062F80895E89462F8089581E090E000C0C2
:10034000EF93FF93EE27E82BE92B31F0E0EAFFE093
:100350003197F1F70197D1F7FF91EF91089501914E
:10036000119121913081089504D00D920020E1F780
:100370000895C8953196002008957F930F93AF9309
:10038000BF938F939F938FB78F938091E20000E884
:10039000081B19F49CB1CBDF12C00091E100A0E66C
:1003A000B0E077279CB1A00FB71F9C9383958093F3
:1003B000E2000395003809F400270093E1008F91D3
:1003C0008FBF9F918F91BF91AF910F917F911895A2
:1003D0007F93AF93BF938F939F938FB78F9390919A
:1003E0006501992399F09A95909365019927A3EE59
:1003F000B0E080916301A80FB91F9C91839580386C
:1004000009F48827809363019CB901C055988F91A6
:100410008FBF9F918F91BF91AF917F911895000FE2
:10042000111F221F331F08950095109520953095B8
:100430000F5F1F4F2F4F3F4F0895019110810BC049
:100440008EDF0BC00191108117FF05C03FEF2FEF2A
:1004500004C0008111272227332737FF03C0E4DFC0
:100460008DE28D93CF92DF92EF92AA24BB24CC240D
:10047000DD24EE2440E2EAE0FF2755E093E38081AB
:10048000890F87FD9F7083FD907F891B81935A950B
:10049000A9F7C5DFAA1CBB1CCC1CDD1CEE1C4A95B1
:1004A00051F7E894EFE0FF2782910CD0EB30E0F7B2
:1004B0001EF068948A2D0AD088278D93EF90DF90E4
:1004C000CF900895982F829501D0892F8F70805DED
:1004D00026F0803309F4089568948D9308950027D9
:1004E0001127222733278D91882339F08053000F5D
:1004F000111F221F331F080FF6CF089588278D93F1
:10050000089509919191992351F08A95D9F73197DE
:10051000002329F081918D930A958823C9F7EECFA6
:100520008FEF83959D919923E1F7089554656D7040
:100530003A20000043002048756D3A200000250055
:040540003100300056
:00000001FF
